:080000000C9406010C940000B1
:100008000C9400000C9400000C9400000C94000068
:100018000C9400000C9400000C9436010C94000021
:100028000C9400000C9440010C9400000C94000007
:100038000C94CA010C9400000C9400000C9400006D
:100048000C9400000C9400000C9400003000310067
:1000580032002E00340035003700380033003600F7
:100068003900B800A600BA00BB00E4007800E5003B
:10007800C0006100B200B300B400BC00BD006F0056
:10008800BE00C100E600C200C3008000E3006500B6
:10009800B600B70070006300BF007900C400C50057
:1000A800C600C700546FC0BA6100546FC0BA6180FF
:1000B800B761BEB86361BD610000A861BCC7BFC4B9
:1000C80080B761BDC7BF61004865BF80E361BDBD42
:1000D800C378000043BF703F00004263B53F000093
:1000E800808080800000A861BCC7BFC480BE7963DF
:1000F800BF6100001027E80364000A000100001037
:100108000001100001004865BF8063B8B4BD61BB41
:100118006100E700220043AC42E04861B365E36553
:10012800BDB865005465BA79E661C780BF6FC0BACB
:10013800613FACB8706FBF613F00E06FBBB46FBF89
:10014800613F7061B770C7B665BD41BABA79BC790D
:10015800BBC7BF6F700025753A25753A2575002510
:1001680075DF0025752E253032750025752E25750D
:100178004D004E0053002575DF2575003A005400E8
:1001880025752E25750080C001002D4E414E0000BA
:100198000B008F020E0101009B021A0101009D0253
:1001A8001C0102009F021E010200A2022001090098
:1001B800A50222010E00AF022C010700BE023A017F
:1001C8000800C60242010800CF024A010B00D8020B
:1001D8005201020060017A01020062017C01020002
:1001E800640184010200660184010200680184013F
:1001F80002006A0186010200A8038E010100AF0314
:1002080090010000F894EE27ECBBF1E0FBBFEBBFD8
:10021800E5BFF8E1F1BDE1BD8DE0A2E0BB27ED93BC
:100228008A95E9F780E094E0A0E6ED930197E9F775
:10023800E8E9F1E085919591009761F0A591B59174
:1002480005901590BF01F00105900D920197E1F717
:10025800FB01F0CFEFE5EDBFE4E0EEBFC0E6D1E093
:100268000C941802EA93EFB7EA93DD24E0E0EEBDC0
:10027800E991EFBFE99118950A921A92AA93BA9355
:10028800EA93FA93EFB7EA93EBB1E871EBB9E03090
:1002980019F4ECB1E0939201E0919101E03011F092
:1002A8000C94C101A0919201A43219F4E1E0E09309
:1002B8006902A0916902A13011F00C94C101E0918A
:1002C8009301A4E9B1E0F0E0EE0FFF1FAE0FBF1FEE
:1002D800E0919201F0E0ED93FC93A0919201AD3092
:1002E80031F0E0919301EF5FE093930146C00E94E3
:1002F8008717E235A0E0FA0761F40E948C17ED3405
:10030800A0E0FA0731F40E949117E334A0E0FA075D
:1003180009F004C0E091B801E0935D020E948717DC
:10032800E734A0E0FA0761F40E948C17E734A0E0F4
:10033800FA0731F40E949117E134A0E0FA0709F0B6
:1003480003C0E1E0E0935C020E948717E734A0E075
:10035800FA0761F40E948C17E335A0E0FA0731F43C
:100368000E949117E635A0E0FA0709F004C00E9440
:100378009617E0936C020E94A617E991EFBFF991D6
:10038800E991B991A9911990099018950A921A9230
:100398006A937A938A939A93AA93BA93EA93FA936D
:1003A800EFB7EA93E4B1F5B10E94AC176627772757
:1003B8000E94061EE0938B02F0938C0260938D02DC
:1003C80070938E02E0918802EF5FE0938802A0911B
:1003D8008802A436E1F40E94AC17E4E6F0E060E09D
:1003E80070E00E94471EE0938902F0938A02EEEAC9
:1003F800E6B9E0E0E0938B02E0938C02E0938D0293
:10040800E0938E02E0938802E1E0E0938702E991AD
:10041800EFBFF991E991B991A99199918991799150
:100428006991199009901895EFEFEBBBE0E0EABBF2
:10043800EFEFE8BBE0E0E7BBEFEFE5BBE0E0E4BBF4
:10044800EFEFE2BBE8E3E1BBE0E8E8B9E4E0E9BFED
:10045800E0E0EFBD0E94B517E0E0EBB9E0E9EAB9EA
:10046800E6E8E0BDE0E0E0BDE3E0E9B9EEEAE6B9E0
:10047800E0E0E7B90E94A41BE0E1EA930E94A01221
:1004880078940E94BA17E0938702EEEEE6B9E091FD
:100498008702E030E1F3A0918902B0918A02A93481
:1004A800E1E0BE0770F40E94BF17E8EDF2E00E9499
:1004B800C5170E94C917EFECF2E00E94C5170E9409
:1004C800CE17829903C0E1E0E0936F02E0E0E09389
:1004D8009101E0935C02E0915C02E030E1F3E0918D
:1004E8005D02E63549F40E9433120E94D617EFE800
:1004F800F2E00E94C517EFC3E13411F00C946F06C7
:10050800E091A201F091A3010E94DC17E091A401FF
:10051800F091A501F097EA0FE0935E02E091A60141
:10052800F091A7010E94DC17E091A801F091A901C0
:10053800F097EA0FE0935F020E949617E09360023B
:10054800E4EEF2E0FA93EA93EEE5F1E0FA93EA9347
:10055800E0915E020E94E217E0915F020E94E217BA
:10056800E09160020E94E2178CE00E9448146096B5
:10057800E091B801F091B9010E94DC17E091BA014D
:10058800F091BB01F097EA0FE0936102E091BC01A2
:10059800F091BD010E94DC17E091BE01F091BF010E
:1005A800F097EA0FE0936202E091C201F091C30173
:1005B8000E94E817E091C401F091C5010E94EF176D
:1005C800E091C601F091C7010E94F717FF93EF93DE
:1005D800E091C801F091C9010E94FF17AF91BF9146
:1005E8000E940B18A3E6B2E00E9412180E94171886
:1005F800E09161020E94E2170E9420180E942518CB
:10060800E09162020E94E2170E942018E2E0F3E003
:100618000E942E180E9435180E943C180E94351816
:100628000E944318E091D201F091D3010E94DC1797
:10063800E091D401F091D501F097EA0FE0936502BB
:10064800E091D601F091D7010E94DC17E091D80122
:10065800F091D901F097EA0FE0936602E091DC018E
:10066800F091DD010E94E817E091DE01F091DF01D1
:100678000E94EF17E091E001F091E1010E94F71765
:10068800FF93EF93E091E201F091E3010E94FF17DD
:10069800AF91BF910E940B18A7E6B2E00E94121812
:1006A8000E944E18E09165020E94E2170E942018ED
:1006B8000E945718E09166020E94E2170E942018D3
:1006C800E0E2F3E00E942E180E9460180E943C1895
:1006D8000E9460180E944318E091EE01F091EF012A
:1006E800F097E0936D02EAE2F3E00E946718E09168
:1006F8006D020E94E2170E942018E091FC01F0911F
:10070800FD01F097A8EEB3E00E942C1EBF01E09116
:10071800FE01F091FF01F097A4E6B0E00E942C1EC4
:100728006E0F7F1FE0910002F0910102F097AAE09E
:10073800B0E00E942C1EDB01AE0FBF1FE091040247
:10074800F0910502F097EA0FFB1FE0936A02F0931D
:100758006B020E946E180E9477180E943C180E9433
:1007680077180E944318EEE3F3E00E946718E091BF
:100778006C020E94E2170E9420180E947E18EEEE7A
:10078800F2E00E94C5170E94D617E8EFF2E00E9437
:10079800C5170E9485180E948B18E6E00E948E18E3
:1007A800E2E0F3E00E94C517EBE00E948E180E9479
:1007B8009318ECE00E948E18E0E6F1E00E94C5175D
:1007C8000E949618ECE0F3E00E94C517E3E00E944F
:1007D8009C18E6E1F3E00E94C517E5E00E949C182A
:1007E8000E948B18E6E00E949C18E0E2F3E00E9469
:1007F800C517EBE00E949C180E949318ECE00E9439
:100808009C18E2E6F1E00E94C5170E94A118E4EEE8
:10081800F2E00E94C517E9E00E94A718E4E3F3E0BC
:100828000E94C517EEE00E948E18EAE2F3E00E94EB
:10083800C517EEE00E949C18EEE3F3E00E94C5178E
:10084800A0E08299A1E0A03021F4A0916F02A1302C
:1008580009F03EC2E0916302F09164020E94AC1874
:100868007F936F93FF93EF93E09162020E94B91810
:100878000E94BF18AF91BF918F919F910E94C81895
:10088800E09161020E94CD18E0937003F093710328
:100898006093720370937303E0916702F0916802AA
:1008A8000E94AC187F936F93FF93EF93E0916602D9
:1008B8000E94B9180E94BF18AF91BF918F919F9164
:1008C8000E94C818E09165020E94CD18E0937C034D
:1008D800F0937D0360937E0370937F03ABEAB1E0EE
:1008E8000E94A21EA0E0B0E088EC92E40E94191DCC
:1008F8007F936F93FF93EF93AFEAB1E00E94A21E3C
:10090800AF91BF918F919F910E94C818E0E0F8ECD9
:100918006FEA78E40E94671D7F936F93FF93EF93CC
:10092800A7EAB1E00E94A21E0E94BF18AF91BF9132
:100938008F919F910E94C91C7F936F93FF93EF93B0
:10094800A3EAB1E00E94A21EAF91BF918F919F913F
:100958000E94C91CADE4B3EF8EE89CE30E94191D08
:10096800E0938003F0938103609382037093830381
:10097800A0917C03B0917D0380917E0390917F03C9
:100988000E94C21CE0939403F0939503609396032E
:10099800709397030E94D7180E94EA16E093840385
:1009A800F093850360938603709387030E94D7189A
:1009B8000E945E16E0938C03F0938D0360938E0380
:1009C80070938F030E94E2180E94EA16E09388034E
:1009D800F093890360938A0370938B030E94E21853
:1009E8000E945E16E0939003F09391036093920344
:1009F800709393030E94ED180E945E160E94F818E7
:100A0800E0939C03F0939D0360939E0370939F0370
:100A18000E94ED180E94EA160E94F818E0939803C5
:100A2800F093990360939A0370939B03E0919C035E
:100A3800F0919D0360919E0370919F03A09188039C
:100A4800B091890380918A0390918B030E94FF18CB
:100A58000E9404197F936F93FF93EF930E940C19E0
:100A68000E9415190E94F8187F936F93FF93EF93D4
:100A78000E9420190E9429190E943419AF91BF9130
:100A88008F919F910E943F190E948B1E0E9404190A
:100A9800AF91BF918F919F910E94C91C0E948B1E9C
:100AA8000E94CC1D7F936F93FF93EF930E940C19C4
:100AB8000E9429190E94F8187F936F93FF93EF9370
:100AC8000E9420190E9415190E943419AF91BF91F4
:100AD8008F919F910E94C91CAF91BF918F919F9157
:100AE8000E944419E093A003F093A1036093A2032A
:100AF8007093A303A6E7BBE782EC9AE40E94191D52
:100B0800A0E7B2E00E94561C0E94731E0E940C19B6
:100B18000E9415190E94F8187F936F93FF93EF9323
:100B28000E9420190E9429190E943419AF91BF917F
:100B38008F919F910E943F19E0937403F09375037E
:100B480060937603709377030E942019A0919C0309
:100B5800B0919D0380919E0390919F030E94191D5F
:100B68000E94231CDF01CB01E0917403F09175030F
:100B780060917603709177030E944419ABE1BFE25C
:100B880085E692E40E94191D0E944A19A0917703F4
:100B9800AA2322F40E9453190E944A190E94531949
:100BA8000E948B1EE0E0F0E064EB73E40E948B1E71
:100BB8000E94C914DF01CB01E0E0F0E064E373E4D4
:100BC8000E943F190E94231C0E944A19A091A70362
:100BD800AA2382F4E091A403F091A5036091A603EF
:100BE8007091A703A0E0B0E084EB93E40E94C91CD5
:100BF8000E944A19A091A403B091A5038091A6036D
:100C08009091A703E0E0F0E068EC72E40E94191DFF
:100C1800A4E7B2E00E941218E2E5F3E0FA93EA933F
:100C2800E6E7F1E0FA93EA93E0917002F09171023D
:100C380060917202709173020E948B1E0E942018AC
:100C4800ECE5F3E0FA93EA93EEE7F1E0FA93EA933E
:100C58000E9462190E943C180E9462190E94691938
:100C68000E943C180E947319E6E6F3E00E94671898
:100C78000E9462190E9469190E946C1EA6E0B0E0E9
:100C88000E942C1E662777270E948B1E0E94201820
:100C9800E0E00E947819ECE5F3E00E94C517E5E072
:100CA8000E9478190E948B18E6E00E947819E6E6FF
:100CB800F3E00E94C517E8E00E9478190E94931893
:100CC800E9E00E947819E2E5F3E00E94C51703C045
:100CD800E0E0E0936F02E0916F02E03081F48299E6
:100CE8000EC00E947D1982990AC00E94BA17E0932B
:100CF8005C020E94A617E1E0E0936E026EC69E9920
:100D08005DC60E947D199E9959C60E94BA17E09344
:100D18005C020E94A6170E948319EF5F0E9488193F
:100D2800E93C60F00E943312E2E00E948E18E2EC87
:100D3800F0E00E948B190E94CE17C8CBE8E4F3E0DC
:100D48000E9467180E9483190E94E2170E942018C7
:100D58000E947E180E948F190E948518E8E4F3E02B
:100D68000E94C517E8E00E948E18E4E6F1E00E94B0
:100D7800C517E0918A01E03011F00C94DC0A0E945A
:100D880092190E949B199A992EC00E947D199A99CE
:100D98002AC0E1E0ED15A9F00E94B5170E94A2193A
:100DA800A1E0A083EFE0EA1520F00E94A7190E94B5
:100DB800AC190E94AF19E1E0DE2EA394E4E0EEBD89
:100DC80012C0AA940E94A219ABE2A083EFE0EA1530
:100DD80030F00E94A719EAE5F0E00E948B190E9402
:100DE800AF19A394DD249B9970C00E947D199B992B
:100DF8006CC0E4E0ED15A1F00E94B517CC240E9468
:100E0800A219A4E0A083EFE0EA1520F00E94A71938
:100E18000E94B5190E94AF19E4E00E94B81955C0A4
:100E2800EC2DE13099F4AA940E94A219AAE0A083BB
:100E3800EFE0EA1530F00E94A719EAE6F0E00E9418
:100E48008B190E94AF19A394C3943FC0E23099F460
:100E5800AA940E94A219ABE0A083EFE0EA1530F053
:100E68000E94A719ECE6F0E00E948B190E94AF19C6
:100E7800A394C3942AC0E33099F4AA940E94A219B7
:100E8800ACE0A083EFE0EA1530F00E94A719EEE687
:100E9800F0E00E948B190E94AF19A394C39415C067
:100EA800E43099F4AA940E94A219ADE0A083EFE07F
:100EB800EA1530F00E94A719E0E7F0E00E948B19CC
:100EC8000E94AF19A394CC24DD249C9970C00E9481
:100ED8007D199C996CC0E7E0ED15A1F00E94B5174B
:100EE800CC240E94A219A7E0A083EFE0EA1520F025
:100EF8000E94A7190E94BF190E94AF19E7E00E943B
:100F0800B81955C0EC2DE13099F4AA940E94A219A1
:100F1800AEE0A083EFE0EA1530F00E94A719E2E7FF
:100F2800F0E00E948B190E94AF19A394C3943FC0AC
:100F3800E23099F4AA940E94A219AFE0A083EFE0EE
:100F4800EA1530F00E94A719E4E7F0E00E948B1937
:100F58000E94AF19A394C3942AC0E33099F4AA94C9
:100F68000E94A219A0E1A083EFE0EA1530F00E94E8
:100F7800A719E6E7F0E00E948B190E94AF19A39425
:100F8800C39415C0E43099F4AA940E94A219A1E16F
:100F9800A083EFE0EA1530F00E94A719E8E7F0E037
:100FA8000E948B190E94AF19A394CC24DD249D992B
:100FB80007C00E947D199D9903C0E1E0E0938A0172
:100FC8000E9492190E94C2199A9970C00E947D19B4
:100FD8009A996CC0E2E0ED15A1F00E94B517CC24F7
:100FE8000E94A219A2E0A083EFE0EA1520F00E9477
:100FF800A7190E94C9190E94AF19E2E00E94B81906
:1010080055C0EC2DE13099F4AA940E94A219A2E1EE
:10101800A083EFE0EA1530F00E94A719EAE7F0E0B4
:101028000E948B190E94AF19A394C3943FC0E23069
:1010380099F4AA940E94A219A3E1A083EFE0EA150B
:1010480030F00E94A719ECE7F0E00E948B190E948B
:10105800AF19A394C3942AC0E33099F4AA940E94C8
:10106800A219A4E1A083EFE0EA1530F00E94A719C5
:10107800EEE7F0E00E948B190E94AF19A394C39485
:1010880015C0E43099F4AA940E94A219A5E1A0839E
:10109800EFE0EA1530F00E94A719E0E8F0E00E94BE
:1010A8008B190E94AF19A394CC24DD249B9970C09E
:1010B8000E947D199B996CC0E5E0ED15A1F00E9496
:1010C800B517CC240E94A219A5E0A083EFE0EA1589
:1010D80020F00E94A7190E94CC190E94AF19E5E0E0
:1010E8000E94B81955C0EC2DE13099F4AA940E94D9
:1010F800A219A6E1A083EFE0EA1530F00E94A71933
:10110800E2E8F0E00E948B190E94AF19A394C394FF
:101118003FC0E23099F4AA940E94A219A7E1A083E3
:10112800EFE0EA1530F00E94A719E4E8F0E00E9429
:101138008B190E94AF19A394C3942AC0E33099F481
:10114800AA940E94A219A8E1A083EFE0EA1530F062
:101158000E94A719E6E8F0E00E948B190E94AF19D7
:10116800A394C39415C0E43099F4AA940E94A219D8
:10117800A9E1A083EFE0EA1530F00E94A719E8E89A
:10118800F0E00E948B190E94AF19A394CC24DD24AF
:101198009C9970C00E947D199C996CC0E8E0ED157F
:1011A800A1F00E94B517CC240E94A219A8E0A08340
:1011B800EFE0EA1520F00E94A7190E94CF190E94BB
:1011C800AF19E8E00E94B81955C0EC2DE13099F448
:1011D800AA940E94A219AAE1A083EFE0EA1530F0D0
:1011E8000E94A719EAE8F0E00E948B190E94AF1943
:1011F800A394C3943FC0E23099F4AA940E94A21920
:10120800ABE1A083EFE0EA1530F00E94A719ECE803
:10121800F0E00E948B190E94AF19A394C3942AC0CE
:10122800E33099F4AA940E94A219ACE1A083EFE0FC
:10123800EA1530F00E94A719EEE8F0E00E948B1939
:101248000E94AF19A394C39415C0E43099F4AA94EA
:101258000E94A219ADE1A083EFE0EA1530F00E94E8
:10126800A719E0E9F0E00E948B190E94AF19A39436
:10127800CC24DD249D992CC00E947D199D9928C0FD
:10128800E4E6ED15A9F00E94B5170E94A219A4E69C
:10129800A083EFE0EA1520F00E94A7190E94D21956
:1012A8000E94AF19E4E6DE2EA394E4E0EEBD10C080
:1012B800AA940E94A219AEE1A083EFE0EA1520F0FB
:1012C8000E94A7190E94D5190E94AF19A394DD2482
:1012D8000E9492190E94D8199A9970C00E947D198B
:1012E8009A996CC0E3E0ED15A1F00E94B517CC24E3
:1012F8000E94A219A3E0A083EFE0EA1520F00E9463
:10130800A7190E94DF190E94AF19E3E00E94B819DB
:1013180055C0EC2DE13099F4AA940E94A219AFE1CE
:10132800A083EFE0EA1530F00E94A719E4E9F0E0A5
:101338000E948B190E94AF19A394C3943FC0E23056
:1013480099F4AA940E94A219A0E2A083EFE0EA15FA
:1013580030F00E94A719E6E9F0E00E948B190E947C
:10136800AF19A394C3942AC0E33099F4AA940E94B5
:10137800A219A1E2A083EFE0EA1530F00E94A719B4
:10138800E8E9F0E00E948B190E94AF19A394C39476
:1013980015C0E43099F4AA940E94A219A2E2A0838D
:1013A800EFE0EA1530F00E94A719EAE9F0E00E94A0
:1013B8008B190E94AF19A394CC24DD249B9970C08B
:1013C8000E947D199B996CC0E6E0ED15A1F00E9482
:1013D800B517CC240E94A219A6E0A083EFE0EA1575
:1013E80020F00E94A7190E94E2190E94AF19E6E0B6
:1013F8000E94B81955C0EC2DE13099F4AA940E94C6
:10140800A219A3E2A083EFE0EA1530F00E94A71921
:10141800ECE9F0E00E948B190E94AF19A394C394E1
:101428003FC0E23099F4AA940E94A219A4E2A083D2
:10143800EFE0EA1530F00E94A719EEE9F0E00E940B
:101448008B190E94AF19A394C3942AC0E33099F46E
:10145800AA940E94A219A5E2A083EFE0EA1530F051
:101468000E94A719E0EAF0E00E948B190E94AF19C8
:10147800A394C39415C0E43099F4AA940E94A219C5
:10148800A6E2A083EFE0EA1530F00E94A719E2EA8D
:10149800F0E00E948B190E94AF19A394CC24DD249C
:1014A8009C9970C00E947D199C996CC0E9E0ED156B
:1014B800A1F00E94B517CC240E94A219A9E0A0832C
:1014C800EFE0EA1520F00E94A7190E94E5190E9492
:1014D800AF19E9E00E94B81955C0EC2DE13099F434
:1014E800AA940E94A219A7E2A083EFE0EA1530F0BF
:1014F8000E94A719E4EAF0E00E948B190E94AF1934
:10150800A394C3943FC0E23099F4AA940E94A2190C
:10151800A8E2A083EFE0EA1530F00E94A719E6EAF6
:10152800F0E00E948B190E94AF19A394C3942AC0BB
:10153800E33099F4AA940E94A219A9E2A083EFE0EB
:10154800EA1530F00E94A719E8EAF0E00E948B192A
:101558000E94AF19A394C39415C0E43099F4AA94D7
:101568000E94A219AAE2A083EFE0EA1530F00E94D7
:10157800A719EAEAF0E00E948B190E94AF19A39418
:10158800CC24DD249D9913C00E947D199D990FC01C
:101598000E94B517AA940E94A219A0E0A0830E94F5
:1015A800A7190E94D5190E94AF19DD24CC24E1CBDC
:1015B800E1E04E2E442049F00E94E8190E94AA1E3C
:1015C8004E2E442009F05394F5CF0E94E819E1E02B
:1015D8000E948819F0E0E653FF4FDF01E52D0E94D5
:1015E800C61E0E94A118EFEAF2E00E94C5170E94E9
:1015F800ED1988248820F1F40E9492190E949B1901
:101608009D9908C00E947D199D9904C0E1E0E0936E
:101618007E028E2E0E9492190E94D8199D9909C0A7
:101628000E947D199D9905C0E2E0E0937E02E1E009
:101638008E2EE0CF8824AA24CC24A0917E02A1304B
:1016480091F50E94F3190E94381AE0916102EA9319
:101658000E94DD1BE0916202EA930E94DD1B0E945A
:1016680035180E94581A0E9435180E945D1AE09198
:101678006502EA930E94DD1BE0916602EA930E94EC
:10168800DD1B0E9460180E94581A0E9460180E9470
:101698005D1A0E9477180E94581A0E9477180E94B3
:1016A8005D1A0E94621AA0917E02A23011F00C9479
:1016B800C40C0E943312E4E00E948E18CC2031F44E
:1016C800EEEBF2E00E94C5170E94ED19E1E0EC157F
:1016D80031F4E6ECF2E00E94C5170E94ED19882467
:1016E800882011F00C948E0C0E9492190E949B196C
:1016F8009A9912C00E947D199A990EC0E7E0EA15DE
:1017080058F00E946A1A0E946D1AA1E0A0830E94F4
:10171800AC190E94AF19A3949B9912C00E947D191D
:101728009B990EC0E7E0EA1558F00E946A1A0E94D9
:101738006D1AA4E0A0830E94B5190E94AF19A39462
:101748009C9912C00E947D199C990EC0E7E0EA1589
:1017580058F00E946A1A0E946D1AA7E0A0830E949E
:10176800BF190E94AF19A3949D992EC00E947D199C
:101778009D992AC0CC2099F40E94721AE0937602AF
:101788000E947C1AE09377020E94861AE0937802FE
:101798000E94901AE0937902AA24C3948ACFE1E0C8
:1017A800EC1591F40E94721AE0937A020E947C1A56
:1017B800E0937B020E94861AE0937C020E94901AB2
:1017C800E0937D02E1E08E2E0E9492190E94C219D8
:1017D8009A9912C00E947D199A990EC0E7E0EA15FD
:1017E80058F00E946A1A0E946D1AA2E0A0830E9413
:1017F800C9190E94AF19A3949B9912C00E947D1920
:101808009B990EC0E7E0EA1558F00E946A1A0E94F8
:101818006D1AA5E0A0830E94CC190E94AF19A39469
:101828009C9912C00E947D199C990EC0E7E0EA15A8
:1018380058F00E946A1A0E946D1AA8E0A0830E94BC
:10184800CF190E94AF19A3949D9912C00E947D19C7
:101858009D990EC0E7E0EA1558F00E946A1A0E94A6
:101868006D1AA0E0A0830E94D2190E94AF19A39418
:101878000E9492190E94D8199A9912C00E947D1943
:101888009A990EC0E7E0EA1558F00E946A1A0E9479
:101898006D1AA3E0A0830E94DF190E94AF19A394D8
:1018A8009B9912C00E947D199B990EC0E7E0EA152A
:1018B80058F00E946A1A0E946D1AA6E0A0830E943E
:1018C800E2190E94AF19A3949C9912C00E947D1935
:1018D8009C990EC0E7E0EA1558F00E946A1A0E9427
:1018E8006D1AA9E0A0830E94E5190E94AF19A3947C
:1018F8009D990FC00E947D199D990BC0AA940E94C2
:101908006D1AA0E0A0830E946A1A0E94D5190E944D
:10191800AF19E6CE0E94F3190E94381AE0917602B8
:10192800EA930E94DD1BE0917702EA930E94DD1B97
:10193800E0917802EA930E94DD1BE0917902EA9334
:101948000E94DD1BE0917A02EA930E94DD1BE09180
:101958007B02EA930E94DD1BE0917C02EA930E94DD
:10196800DD1BE0917D02EA930E94DD1BE0E0EA9333
:101978000E94DD1BE0E0EA930E94DD1B0E94621AD0
:101988000E9433120E949618E2EBF0E00E948B1935
:101998000E94CE17AA24E4E1AE1630F40E94A219E0
:1019A800A0E0A083A394F7CFAA24DD24CC24552457
:1019B8008824E0E0E0937E02E0938A019F99F9C4CD
:1019C8000E947D199F99F5C40E94BA17E09393016C
:1019D800E0E0E0935C02E09369020E948319E03042
:1019E80061F40E9433120E94BF17E0EDF0E00E94FC
:1019F8008B190E94CE170C946A020E943312E2E0FF
:101A08000E948E180E948F19E7E00E948E18E6E661
:101A1800F1E00E94C5178824882011F00C94250E47
:101A28000E9492190E949B199A9912C00E947D19CE
:101A38009A990EC0E2E0EA1558F00E949A1A0E949C
:101A4800A219A1E0A0830E94AC190E94AF19A39427
:101A58009B9912C00E947D199B990EC0E2E0EA157D
:101A680058F00E949A1A0E94A219A4E0A0830E942A
:101A7800B5190E94AF19A3949C9912C00E947D19B0
:101A88009C990EC0E2E0EA1558F00E949A1A0E944A
:101A9800A219A7E0A0830E94BF190E94AF19A394BE
:101AA8009D9929C00E947D199D9925C0EA2DE13094
:101AB80019F4B09076011DC0E23049F4E091760146
:101AC800AAE0EA9FF001AE2FE091770110C0E33061
:101AD80081F4E0917601A4E6EA9F602DE091770118
:101AE800AAE0EA9FF001A62FAE0FE0917801EA0F75
:101AF800BE2EE1E08E2E0E9492190E94C2199A9978
:101B080012C00E947D199A990EC0E2E0EA1558F0B9
:101B18000E949A1A0E94A219A2E0A0830E94C919E1
:101B28000E94AF19A3949B9912C00E947D199B999A
:101B38000EC0E2E0EA1558F00E949A1A0E94A21913
:101B4800A5E0A0830E94CC190E94AF19A3949C9988
:101B580012C00E947D199C990EC0E2E0EA1558F067
:101B68000E949A1A0E94A219A8E0A0830E94CF1985
:101B78000E94AF19A3949D9912C00E947D199D9946
:101B88000EC0E2E0EA1558F00E949A1A0E94A219C3
:101B9800A0E0A0830E94D2190E94AF19A3940E94CA
:101BA80092190E94D8199A9912C00E947D199A997F
:101BB8000EC0E2E0EA1558F00E949A1A0E94A21993
:101BC800A3E0A0830E94DF190E94AF19A3949B99F8
:101BD80012C00E947D199B990EC0E2E0EA1558F0E8
:101BE8000E949A1A0E94A219A6E0A0830E94E219F4
:101BF8000E94AF19A3949C9912C00E947D199C99C8
:101C08000EC0E2E0EA1558F00E949A1A0E94A21942
:101C1800A9E0A0830E94E5190E94AF19A3949D9999
:101C28000FC00E947D199D990BC0AA940E94A21909
:101C3800A0E0A0830E949A1A0E94D5190E94AF19A9
:101C4800EBCE0E947D190E943312AA24E4E1AE165D
:101C580030F40E94A219A0E0A083A394F7CFAA248D
:101C68000E948319EB15A8F40E94BF17E0EDF0E07D
:101C78000E948B190E94CE17E2E00E948E180E94E3
:101C88008F19E7E00E948E18E8E6F1E00E94C51778
:101C9800C2CE0E943312E8E4F3E00E946718EB2DED
:101CA8000E94E2170E942018E0E00E948E18EAE6DF
:101CB800F1E00E94C517E1E00E948E18E8E4F3E025
:101CC8000E94C5170E949D1AE695E6957E2E0E94F1
:101CD8009D1AE295E07FEE0FEE0F6E2EAA24E0E14A
:101CE800AE1610F00C94CB0F0E94A41A0E94A219F1
:101CF800FF93EF930E94B61AAF91BF91EC930E94A5
:101D0800B81B0E94A219E081E03029F40E94A719AB
:101D1800E2E9F0E033C1E13029F40E94A719E6E5D1
:101D2800F0E02CC1E23029F40E94A719E8E5F0E0C0
:101D380025C1E33029F40E94A719E4E6F0E01EC1AA
:101D4800E43029F40E94A719ECE5F0E017C1E5306A
:101D580029F40E94A719EEE5F0E010C1E63029F455
:101D68000E94A719E6E6F0E009C1E73029F40E94CD
:101D7800A719E0E6F0E002C1E83029F40E94A719AB
:101D8800E2E6F0E0FBC0E93029F40E94A719E8E692
:101D9800F0E0F4C0EB3229F40E94A719EAE5F0E07C
:101DA800EDC0EA3029F40E94A719EAE6F0E0E6C09F
:101DB800EB3029F40E94A719ECE6F0E0DFC0EC3024
:101DC80029F40E94A719EEE6F0E0D8C0ED3029F416
:101DD8000E94A719E0E7F0E0D1C0EE3029F40E9494
:101DE800A719E2E7F0E0CAC0EF3029F40E94A7196A
:101DF800E4E7F0E0C3C0E03129F40E94A719E6E760
:101E0800F0E0BCC0E13129F40E94A719E8E7F0E04E
:101E1800B5C0E23129F40E94A719EAE7F0E0AEC0A4
:101E2800E33129F40E94A719ECE7F0E0A7C0E431F8
:101E380029F40E94A719EEE7F0E0A0C0E53129F4E3
:101E48000E94A719E0E8F0E099C0E63129F40E9461
:101E5800A719E2E8F0E092C0E73129F40E94A71937
:101E6800E4E8F0E08BC0E83129F40E94A719E6E81D
:101E7800F0E084C0E93129F40E94A719E8E8F0E00D
:101E88007DC0EA3129F40E94A719EAE8F0E076C09B
:101E9800EB3129F40E94A719ECE8F0E06FC0EC31AF
:101EA80029F40E94A719EEE8F0E068C0ED3129F4A2
:101EB8000E94A719E0E9F0E061C0EE3129F40E9420
:101EC800A719E2E9F0E05AC0EF3129F40E94A719F6
:101ED800E4E9F0E053C0E03229F40E94A719E6E9EA
:101EE800F0E04CC0E13229F40E94A719E8E9F0E0DB
:101EF80045C0E23229F40E94A719EAE9F0E03EC0A1
:101F0800E33229F40E94A719ECE9F0E037C0E43283
:101F180029F40E94A719EEE9F0E030C0E53229F46F
:101F28000E94A719E0EAF0E029C0E63229F40E94ED
:101F3800A719E2EAF0E022C0E73229F40E94A719C3
:101F4800E4EAF0E01BC0E83229F40E94A719E6EAA7
:101F5800F0E014C0E93229F40E94A719E8EAF0E099
:101F68000DC0E43629F40E94A719E4E5F0E006C0A4
:101F7800EA3251F40E94A719EAEAF0E0FA93EA93E8
:101F88000E947F120E94BA1A6394A394A8CEAA242E
:101F9800E4E1AE1630F40E94A219A0E0A083A39455
:101FA800F7CFAA24E0916E02E03011F00C9498105B
:101FB800AA24EAE0AE1690F40E94A41A0E94C01A5D
:101FC800FF93EF930E94B61AAF91BF91EC930E94D2
:101FD800B81B0E94BA1A6394A394EBCF0E941718F7
:101FE800E0916C010E94E2170E9420180E942518B7
:101FF800E0916D010E94E2170E942018E2E0F3E0F0
:102008000E94C51AE0916E010E94E217E0916F01EB
:102018000E94E2170E9473190E944E18E091700105
:102028000E94E2170E9420180E945718E09171013F
:102038000E94E2170E942018E0E2F3E00E94C51A0D
:10204800E09172010E94E217E09173010E94E21789
:102058000E9473190E946E18E09174010E94E217A1
:10206800E09175010E94E2170E947319E1E00E9455
:10207800A718EEEEF2E00E94C517E4E00E94A71848
:10208800E8EFF2E00E94C517E6E00E94A7180E9458
:102098008B18E7E00E94A718E2E0F3E00E94C5175A
:1020A800ECE00E94A7180E949318EDE00E94A71880
:1020B800EFE9F2E00E94C517E1E00E947819ECE030
:1020C800F3E00E94C517E4E00E947819E6E1F3E026
:1020D8000E94C517E6E00E9478190E948B18E7E075
:1020E8000E947819E0E2F3E00E94C517ECE00E9434
:1020F80078190E949318EDE00E947819E2EAF2E05C
:102108000E94C5170E948518E4E3F3E00E94C517F2
:10211800AA24EAE0AE1630F40E94C01AA0E0A08318
:10212800A394F7CFAA2433C0E13089F5AA24E8E0C4
:10213800AE16D8F40E94A41AEA2DA3E9B1E0F0E0A3
:102148000E94171EEA0FFB1FFF93EF930E94B61A17
:10215800AF91BF910E94B9180E94B61E0E94B81B89
:102168000E94BA1A6394A394E2CFAA24E3E00E94DF
:10217800A718E5EAF2E00E94C517E0E0E0936E02D6
:10218800E1E0E0936F020E94CE170C946A02992452
:10219800992011F00C9462110E9492190E94D8198A
:1021A8009D9922C00E947D199D991EC0A091900101
:1021B800A13021F0A0918E01A13079F4E0E0E09304
:1021C8009001E0938E01ECE00E948E18E8EEF0E0BA
:1021D8000E948B190E94ED1907C00E943312E2B3C6
:1021E800E863E2BBE1E09E2E0E9492190E94C219A8
:1021F8009A990BC00E947D199A9907C0B3940E94BE
:102208008319EB1508F045CDBA949D990AC00E9430
:102218007D199D9906C0BA94E0E0EB1508F439CD14
:10222800B3940E9492190E949B199D992DC00E94F7
:102238007D199D9929C0E0919001EF5FE09390018D
:10224800E130C9F4A0918E01A13059F4E1E0E093A6
:102258008F01E0E0E0938E01E0939001E1E09E2E93
:1022680009C0ECE00E948E18ECEDF0E00E948B199A
:102278000E94ED1909C0E23039F4E1E0E0938D01E4
:102288009E2EE0E0E09390019A9917C00E947D1974
:102298009A9913C0A0919001A13079F4E1E0E093FC
:1022A8008E01E0E0E0939001ECE00E948E18E2EEEF
:1022B800F0E00E948B190E94ED196ACFA0918D0160
:1022C800A13011F00C94B411AB2DB0E0AF5FBF4F4B
:1022D800E0E00E94C61EEB2DF0E0E0938B01F09346
:1022E8008C010E9483190E94CC1AF0E0AE17BF0738
:1022F800B0F4E0918B01F0918C01E653FF4F0F0190
:10230800E0918B01F0918C01E553FF4FDF010E94B2
:10231800AA1ED0010E94C61E0E94D11AE2CF0E94B6
:10232800D91A0E948319E1500E948819E03079F483
:102338000E9433120E94C917EEEEF0E00E948B193A
:102348000E94CE17E0E0E0938D010C946A020E948F
:102358008319EB1508F4BA94E0E0E0938D0199CC69
:10236800A0918F01A13029F50E94D91A0E94CC1A98
:10237800A93CE0E0BE0750F40E94CC1AAF5FBF4F03
:10238800E0E00E94C61E0E94D11AF0CF0E94D91A1E
:10239800E0E0E0938F01A0E0B0E00E94C61E0E943A
:1023A80033120E94C917EEEEF0E00E948B190E94CA
:1023B800CE170C946A02FFCFFFE0FA95F1F7089563
:1023C800A7B3AF70A7BBC19AC098F6DFC29AF4DF73
:1023D800A6B3C298F1DFC29AEFDFC298A7FDF5CF86
:1023E8000895A07FAB2BA8BBC29A0E94E011C298A7
:1023F8000E94E0110895C198A7B3A76FA7BBB8B30F
:10240800BF70A881EEDFA881A295EBDFC19A0C947A
:10241800D312C29A0E94E011E6B3C2980E94E0115A
:10242800E07F08950E94E011F4DFAE2FF2DFC1983B
:10243800E295EA2B08950E94E411E881F0E0E8555E
:10244800FC4FE081A981EA0FEA930E94FF11E9811C
:10245800E093AC03E881E093AD03229608950E94CF
:10246800E411E2E0EA930E94FF110E94E411ECE01B
:10247800EA930E94FF110E94E411E1E0EA930E94AE
:10248800FF11E0E0E093AD03E093AC030895EF9310
:10249800FF93A8816894AA3039F0E894E091AE03DC
:1024A800A091AC03AE1760F0E091AD03EF5FE0934D
:1024B800AD03E0E0EA93E091AD03EA93BCDF56F0A8
:1024C800E091AC03EF5FE093AC037ADFC09AA88198
:1024D800AA9391DFFF91EF910C94D3121A93A981DB
:1024E800BA81ED91A983BA831E2FE03019F01A93AF
:1024F800CEDFF5CF0EC01A93E981FA813196E983D0
:10250800FA833197E4911E2FE03019F01A93BFDF58
:10251800F3CF188123960895AA27BB271197F1F7BF
:102528000895C198A7B3A76FA7BBB8B3BF70A88118
:102538000E94F511C19A33C0C298C098E881E0930F
:10254800AE03E058E093AA03E881E054E093AB03BC
:102558000E94DF1A0E94DF1A0E94DF1ADDDFE0E224
:10256800EA93DFDFD9DFE8E20E94E51AE4E00E949F
:10257800E51AE5E80E94E51AA7B3AF70A7BBC19AB0
:102588000E941612E53011F0E0E009C00E94E41143
:10259800E6E0EA930E94FF110E943312E1E02196DF
:1025A80008951A930A93AA81BB8112960E946F1EFE
:1025B800309759F1AA81BB8114960E946F1E8F0132
:1025C800309761F00230E0E01E07F0F0F801319733
:1025D8008F01AA81BB811496ED93FC93AA81BB81DC
:1025E8001296ED91FD913196FE93EE933197AC8161
:1025F800A083AA81BB810E946F1EFF232AF0ED9160
:10260800FD913196FE93EE9306C0AA81BB81EFEF50
:10261800FFEFED93FC93198108812596089526977D
:102628000E94E61E10E0AC85BD85E0E0F0E0ED9389
:10263800FC93EA89FB893196EA8BFB8B3197E4910D
:102648002E2FE03011F40C944014E12FE03039F4CF
:10265800253211F411E002C00E94EA1A0CC1E130DF
:10266800A9F4253219F40E94EA1A04C112E040E0E4
:1026780000E02D3211F401E0FEC02B3211F44BE2E0
:10268800FAC0203211F440E2F6C002C0E23039F458
:1026980050E013E0203311F40068EDC004C0E330CB
:1026A80011F00C943F14203310F02A3308F007C0BF
:1026B800AAE05A9F502DE22FE0535E0FDCC0E22FB4
:1026C800E33649F40E94F31AE889F989A481AA93A8
:1026D8000E94F91ACFC0E33741F40E94F31A0E940E
:1026E800011B0E9472171E2F0AC0E03761F40E9476
:1026F800F31A0E94011B0E947C171E2F08600260BB
:102708000F7730E035C0E43611F0E93611F4046093
:1027180002C0E53731F4ECEFF0E0EE83FF8315E01B
:102728000DC0E83511F4086004C0E83711F00C94C6
:102738003E14E6E0F1E0EE83FF8314E002FF14C0EC
:102748000E94F31A0E940B1BAB85AA233AF4EA8570
:10275800FB850E940B1EEA87FB874DE2403011F093
:102768001F5F01C00B7F04C00E94F31A0E940B1B5D
:1027780000FD11C0151778F407FF08C002FF04C058
:102788000B7F242F115001C020E301C020E20E94DA
:10279800EA1A5150EFCF312F01FF17C03030A1F0A6
:1027A80003FF06C0EE81FF812591EE83FF8305C0FC
:1027B800AE81BF812D91AE83BF830E94EA1A50304B
:1027C80009F051503150EACF4BC020E3EE81FF8130
:1027D8000E94781EE887F987EE81FF813296EE83A2
:1027E800FF83E885F985AA85BB85AE17BF0750F03A
:1027F8002F5FA885B985EA85FB85EA1BFB0BEA876D
:10280800FB87EFCF2A3328F003FF02C0295F01C0FE
:10281800295D04FD1AC0213320F4A885B9851197D4
:1028280009F409C0531710F000FF01C013C020E2DB
:1028380007FF0BC020E3006102FF07C00B7F4A932C
:102848000E94F91A503009F051500E94EA1A50308B
:1028580009F051503150A885B985129708F0B5CFC5
:1028680000FF08C0503031F05150E0E2EA930E9476
:10287800F91AF8CF10E0DDCEAC85BD850E946F1E39
:102888000E94ED1E64960895FF92F82E26970E94E6
:10289800E81E0E94131B309719F4EFEFFFEF25C0D5
:1028A800DE0116960E94021E8D010E94131BEE8304
:1028B800FF83E0E0E887E987DE011A960E94021E9E
:1028C8000E946F1EFA93EA931A930A93E5EDF2E1D8
:1028D800FA93EA93FE013A96FA93EA93A0DE9F01EF
:1028E800AE81BF81E0E0EC93F9010E94EF1E2A96C9
:1028F800FF9008957B816A81F981E88177FB770FE2
:1029080067FD7160972F9E5781F078F0983190F4A9
:10291800AA27BB27882708948795B795A7959A95DE
:10292800D1F7EA23FB23682305C0E8947727EE272D
:10293800FF2766276F77769508F4606877F9A9917D
:10294800B99189919991EA17FB076807790797FB6D
:1029580008950E941A1B0E941D1B19F40E941A1B3D
:10296800BBC2E6F70E94241B0E94C21CB5C20E948B
:102978001A1B0E941D1B19F40E941A1BADC2E6F314
:102988000E94241B0E94C91CA7C224970E942A1BCC
:102998000E94D71E19F40E942F1B8AC10E942A1B6D
:1029A8000E94341B0E94671D0E94391B0E94D71E7B
:1029B80019F40E942F1B7CC10E943C1B0E94DB1E45
:1029C80024F40E943F1BC5DF03C00E943F1BCFDFDA
:1029D8000E94861E0E941A1B0E94431B0E94191DFA
:1029E8000E94341B0E943F1963C124971A930A93CB
:1029F8000E94481B0E94DB1E2CF0EFEFFFEF6FE7F1
:102A08007FEF73C00E944D1B0E948B1EEDB7FEB76F
:102A18003197FA93EA931F930F930E94021C0F9128
:102A28001F910E94521B0E94481BE3EFF4E065E3EC
:102A38007FE30E94AC1D40F40E94571B0E94C91CF2
:102A48000E94521B015010400E94591B0E94C21C38
:102A58007F936F93FF93EF930E94591B0E94C91CA9
:102A6800AF91BF918F919F910E94671D0E94521B49
:102A78000E94571B0E945F1BA6E2B2E485E69FE313
:102A88000E94191DDF01CB01EEE4F1E164E570E479
:102A98000E943F190E94481B0E94191D7F936F9343
:102AA800FF93EF930E94661BADE4B1E184ED9FE3D1
:102AB8000E94C21CAF91BF918F919F910E94671D88
:102AC8007F936F93FF93EF93F8010E94221E0E9459
:102AD8008F1CA8E1B2E781E39FE30E94191DAF9123
:102AE800BF918F919F910E94C91C198108812A96D4
:102AF800089528971A930A930E946B1BE0E5FCEA55
:102B08006EEA72EC0E94AC1D18F40E942F1B84C060
:102B1800EA85FB856C857D850E94D71E29F4E0E057
:102B2800F0E060E87FE378C00E946B1BE8E1F2E721
:102B380061EB72E40E94AC1D09F010F40C94A91525
:102B4800EFEFFFEF6FE77FE767C00E946B1BEBE3D8
:102B5800FAEA68EB7FE30E94191DEA87FB876C8716
:102B68007D870E948B1EF5DE0E94581C8F01F8019C
:102B78000E946B1B0E94221E0E948F1C0E943F19FC
:102B8800DF01CB010E94701B0E943F190E94521B5B
:102B98000E94571B0E945F1BADE6BCE48CE69DE3D8
:102BA8000E94191DA6EAB3EE86EE90E40E94C91CA5
:102BB8000E94481B0E94191D0E94521B0E94661BFE
:102BC800A8E2BDE886EA91E40E94C91CEA83FB8377
:102BD8006C837D830E944D1BAA81BB818C819D8162
:102BE8000E94C91CA3EFB4E085EB9FE30E94191D66
:102BF8007F936F93FF93EF930E94481B0E94661B7D
:102C08000E94C21CAF91BF918F919F910E94751B2A
:102C18001A930A930E94151C198108812E9608950B
:102C280024970E947A1B0E94D71E19F40E942F1B1A
:102C38003FC00E94341B0E94DB1E84F40E942A1BA2
:102C48000E94D71E29F4E0E0F0E060E87FE330C09E
:102C58000E947A1B0E947F1B4CDF2AC00E942A1BFD
:102C6800DE010E94581C0E94731E0E941A1B0E94BB
:102C78008F1CDF01CB010E942A1B0E94E11E19F064
:102C88000E942F1B15C00E947A1B0E94231C0E94C1
:102C98007F1B2FDFE887F9876A877B87E881E170E8
:102CA80019F40E947A1B04C00E947A1B0E94231CFC
:102CB8002C96089524971A9310E00E94851BE3E848
:102CC800F9EF62E27EE30E94191D0E948A1B0E94AE
:102CD8008F1B0E948B1E3DDE0E94851B0E943F19A0
:102CE8000E948A1B0E94851B0E94701B0E94AC1DBB
:102CF80009F010F40C948B160E948F1BA0E0B0E032
:102D080080E09FE30E94C21C0E948A1B11E00E947F
:102D1800851BE0E0F0E060E87EE30E94AC1D09F06E
:102D280010F40C949F160E94851B0E94701B0E9431
:102D3800C21C0E948A1B103031F00E948F1B0E9417
:102D4800231C0E948A1B0E948F1B0E94851B0E94C5
:102D5800191DE983FA836B837C83A1EBB4EC86E2CB
:102D680092E40E94191DDF01CB01EDE1F5EE6DE261
:102D780072E40E943F190E94941BACE4B3E584E01E
:102D880091E40E94C91C0E94851B0E94191D7F9313
:102D98006F93FF93EF93E981FA816B817C81A1E1C5
:102DA800BDEE8EED9FE30E94C91C0E94941BAEE508
:102DB800BBE788EA9FE30E94C91CAF91BF918F913E
:102DC8009F910E94671D1881299608950E943C1BB7
:102DD800EBEDFFE069EC7FE30E94C21C0E948B1EB2
:102DE80069DF7AC024970E942A1B0E94431B0E9415
:102DF800191D0E94391BA5E6B0ED8BEC90E40E94EA
:102E08009B1B0E94431B0E94191D7F936F93FF9386
:102E1800EF930E941A1BA0E0BDE689E291E40E94AC
:102E2800C91C0E943C1B0E949B1BAF91BF918F91B4
:102E38009F910E94671D289608950E943C1BEDEC07
:102E4800F3E164ED7EE30E94AC1D20F40E943F1B79
:102E5800C9DF42C00E943C1BEAE7F2E86AE170E47D
:102E68000E94AC1D09F010F40C9446170E94241B14
:102E78000E94751BB7DFABEDBFE089EC9FE30E94B2
:102E88003F192AC00E94241B0E94C21C7F936F9383
:102E9800FF93EF930E94241B0E94C91CAF91BF911E
:102EA8008F919F910E94751B9DDFABEDBFE089E478
:102EB8009FE30E94C91C10C0AB81AA2322F00E9484
:102EC8003F1BBBDF09C00E941A1B0E94231C0E94E3
:102ED8008B1EB3DF0E94231C24960895A991B991F3
:102EE800EE27FF276D91662311F03196FBCF0895E9
:102EF800AA27BB27E991F9910590002011F01196B6
:102F0800FBCFFD010895E0919A01F0919B0108958E
:102F1800E0919C01F0919D010895E0919E01F0914E
:102F28009F010895E091AA01F091AB01F097AAE002
:102F3800EA9FF001AE2FE091AC01F091AD01F0975E
:102F4800EA0F0895E0E0E0939301E09369020895A1
:102F5800A0918B02B0918C0280918D0290918E028B
:102F68000895E0E0EEBDEDBDECBD0895E1E0E0932D
:102F78009101E0E00895E2E0EA93E1E0EA930C943D
:102F88001F12FA93EA930C947212E2E0EA93EA931E
:102F98000C941F12E0EDF7E0FA93EA930E94F61BF7
:102FA8000C943312E3E0EA93E0E0EA930C941F12E6
:102FB800F097AAE0EA9FF001AE2F0895FF27662751
:102FC80077270E948B1E0895F097A8E5B2E00E942B
:102FD8002C1EBF010895F097ACE3B0E00E942C1EB0
:102FE8006E0F7F1F0895F097A6E0B0E00E942C1E98
:102FF800E60FF71F0895F097662777270E948F1C22
:10300800AAE9B9E989E19FE30E94191D0895882773
:1030180099270E94921E0E94C91C08950E94561C5E
:10302800ED93FC930895EEEEF2E0FA93EA93E7E667
:10303800F1E0FA93EA93089584E00E9448142896F0
:103048000895E8EFF2E0FA93EA93E4E6F1E0FA9300
:10305800EA930895FA93EA93EBE6F1E0FA93EA9398
:103068000895A0916302B0916402E4E6F0E0089547
:103078000E94341E662777270E948B1E08950E949F
:103088006C1E662777270E948B1E88E00E944814D2
:103098002C960895ECE0F3E0FA93EA93E7E6F1E082
:1030A800FA93EA930895E6E1F3E0FA93EA93E4E603
:1030B800F1E0FA93EA930895A0916702B09168024B
:1030C800E4E6F0E00895FA93EA93E4E6F1E0FA938F
:1030D800EA930895E4E3F3E0FA93EA93E3E7F1E08F
:1030E800FA93EA930895A0916A02B0916B02EAE01C
:1030F800F0E008950E943312E0E0EA93EA930C941A
:103108001F12E5E0EA93E0E0EA930C941F12EBE962
:10311800F2E037CFEA93E0E0EA930C941F12EDE96E
:10312800F2E02FCFE0E0EA93E1E0EA930C941F127B
:10313800EA93E1E0EA930C941F12E0E0EA93E2E0FC
:10314800EA930C941F12EA93E2E0EA930C941F129C
:10315800662777270E948F1CDF01CB01E0E0F8EC9F
:103168006FEA78E40E94671D0895FF27662777278E
:103178000E948F1C0895DF01CB01E0E0F0E060E7DA
:1031880072E40E94671D08950E94C91CDF01CB01EB
:103198000895EBDF0E94C91CADE4B3EF8EE89CE311
:1031A8000E94191D0895E0917003F09171036091D8
:1031B8007203709173030E948B1E0895E091780347
:1031C800F091790360917A0370917B030E948B1EC2
:1031D8000895E0919403F09195036091960370919E
:1031E80097030E948B1E0895A0E0B0E48CE196E45A
:1031F8000E94191D08950E94191D0E948B1E089592
:10320800E0E0F0E060E070E40E948B1E0C9414167D
:10321800E0919003F0919103609192037091930370
:103228000895A0918403B0918503809186039091BD
:1032380087030E94191D0895E0918803F09189037E
:1032480060918A0370918B030895A0918C03B091CB
:103258008D0380918E0390918F030E94191D08950C
:10326800A0919803B091990380919A0390919B0340
:103278000E94191D08950E94951E0E94C21C08955F
:103288000E94671D0E948B1E0C946017E093A40394
:10329800F093A5036093A6037093A7030895E091A4
:1032A800A403F091A5036091A6037091A703A0E081
:1032B800B0E084E393E40E94C91C0895A0917402CD
:1032C800B0917502E4E6F0E008950E946C1EA6E055
:1032D800B0E00E942C1EDF01EAE0F0E0089588E0EB
:1032E8000E9448142C960895EA93E3E0EA930C941C
:1032F8001F12E2E3F0E0FA93EA930C94F61BA0E0C5
:10330800B0E00E94AA1E08950E94C61EF8CFFA9344
:10331800EA930C947F12ECEAF0E0F9CFE2B3E863A9
:10332800E2BBE5E0F0E0FA93EA930C94F61B95987B
:10333800E5E0F0E0FA93EA930C94F61BEA2DF0E04E
:10334800EA58FE4F0895AA92E1E0EA930C941F12FE
:10335800E6E5F0E0DCCFECE2F1E0FA93EA930C94D6
:10336800F61BECE5F0E0D3CFDE2EE1E0CE2EA39401
:10337800E4E0EEBD0895E0E6F0E0C9CF9498E5E01A
:10338800F0E0FA93EA930C94F61BE8E5F0E0BFCF7F
:10339800EEE5F0E0BCCFE2E6F0E0B9CFE4E5F0E03E
:1033A800B6CFE2E9F0E0B3CF9398E5E0F0E0FA9326
:1033B800EA930C94F61BE4E6F0E0A9CFE6E6F0E029
:1033C800A6CFE8E6F0E0A3CFA52DB0E0AF5FBF4FF2
:1033D8000895E4EFF1E0FA93EA930C94F61B0E9447
:1033E800A91BE0EAEA930E94DD1BE52DE695E69528
:1033F800EA930E94DD1BE52DE295E07FEE0FEE0FCC
:10340800EA930E94DD1BE0917601EA930E94DD1B9E
:10341800E0917701EA930E94DD1BE0917801EA933D
:103428000E94DD1BE0917901EA930E94DD1BE09187
:103438007A01EA930E94DD1BE0917B01EA930E94E6
:10344800DD1BE0917C01EA930E94DD1BE0917D0188
:10345800EA930E94DD1BE0917E01EA930E94DD1B46
:10346800E0917F01EA9308950E94DD1BE0918001BD
:10347800EA930E94DD1BE0918101EA930E94DD1B23
:10348800E0918201EA930E94DD1BE0918301EA93B7
:103498000E94DD1BE0918401EA930E94DD1BE0910C
:1034A8008501EA930C94DD1B0E94341EEA930C9468
:1034B800DD1B0E946C1EEA930C94DD1B0E94B81B56
:1034C800EAE0F0E0FA93EA930C94F61BEA2DEC5F3D
:1034D8002FCEEA2DF0E0E158FD4F0895E0917F02EC
:1034E800AAE0EA9FF001AE2FE0918002EA0F08956A
:1034F800E0918102AAE0EA9FF001AE2FE0918202FA
:10350800EA0F0895E0918302AAE0EA9FF001AE2F46
:10351800E0918402EA0F0895E0918502AAE0EA9F0B
:10352800F001AE2FE0918602EA0F0895EA2DE85FD8
:10353800F1CDAB2DB0E0A653BF4F0E94AA1E08954F
:103548000E94A91BE0EAEA930E94DD1B7A920E947E
:10355800DD1B6A920E94DD1B0E94A91BE1EAEA9327
:103568000C94DD1BE0E0EA930C94C21BE5E0F0E06C
:10357800FA93EA930C94F61BEA2DF0E0E459FE4F17
:103588000895FA93EA93E8E8F1E0FA93EA93089544
:10359800A0918B01B0918C010895ABE8B1E0ED9159
:1035A800FD913196FE93EE930895E0E0E0938B0150
:1035B800E0938C0108950E949012E0E3EA930C9442
:1035C8009512EA930E94FF110C9490122A93ED85AC
:1035D800FE85FA93EA93E989FA8909950895E889B5
:1035E800F9893497E88BF98B0895ED85FE85FA9370
:1035F800EA93E989FA8909950895A889B9891496F9
:103608000E946F1EEE83FF83FA93EA930895A889B8
:10361800B98914960E946F1EEA87FB870895DE0118
:103628001C960E94021E0E946F1E08950E947C1E16
:1036380008950E948B1E0E947E140E94861E089583
:10364800F5DFA0E0B0E080E89FE30895EC81FD811C
:103658006E817F810895E0E0F0E060E070E0089519
:10366800A885B9858A859B8508950E94861EDECF28
:103678000E94811E0895DADF0E948B1E0895AC8196
:10368800BD818E819F810895AE81BF81888599858E
:103698000895EE81FF81688579850895EE83FF831B
:1036A800688779870895F5DFEFCFF3DFA0E0B0E012
:1036B80080E89FE308950E94191DEA83FB836C83C9
:1036C8007D830895EA81FB816C817D810895AA85B7
:1036D800BB858C859D850895E0E0F0E060E07FE3A0
:1036E80008950E94671D0E948B1E0895E885F9853C
:1036F8006A857B8508950E948B1E0E94F914BFDF9E
:103708007ACDAD81BE818F8198850895ED83FE8342
:103718006F8378870895ED81FE816F81788508959C
:10372800A981BA818B819C810E94191D08950E94EC
:10373800191DAEE4BFE88AE491E40E94C91C08950B
:10374800A898A998A09AA19815C0A198A098EE2722
:103758000000999B0895989B089504D0A19A02D0DF
:10376800A09AE1E06CE007C0A19AA09A03D0A098C3
:10377800F9DFA19869E16A95F1F7089578E0A098D2
:10378800F1DF989BFECFEEDF889499990894A09A70
:10379800F1DFEE1F7A9599F77991772311F4A198C3
:1037A80001C0A19ADFDFA098E5DFA09ADBDFA1982E
:1037B800D9CFE99178E0EE0F10F4A19801C0A19A51
:1037C800D9DFA098CFDF989BFECFCCDFA09A7A955F
:1037D80091F7A198C7DFA098CDDFE1E09999EE278E
:1037E800A09AC0CFE991F991309639F083E397E038
:1037F8000197F1F7A8953197C9F70895A991B9915B
:10380800E991F9916991799177FB660F771F88277C
:103818007E57880B7D938C937EE7769567957EF02F
:103828000895A991B991E991F9916991799177FBF5
:10383800660F771F7A0F769567950EF00895309783
:103848006040704009F070580895552342F450388C
:1038580011F4E0FF04C03196691F791F6BF050E83E
:10386800572711F45F93CFC05F3F31F0660F000C0C
:1038780057956795752F08955F9300200AF0CFC07C
:10388800C8C050E8192E1522880F991F9527550F83
:10389800879550E8072E0522660F771F7527550F65
:1038A80067950895689401C0E8945F93F2DF7038D3
:1038B80018F07F3F08F4A7C056E1571BAAF45195AA
:1038C80058300EF4593030F0EFEFFFEF6FEF7FE72D
:1038D80077F91AC077275523B9F0EE0FFF1F661F37
:1038E800771F5A95D1F710C07727583028F0EF2F57
:1038F800F62F672F5850F9CF552331F076956795F5
:10390800F795E7955A95D1F700200AF484D15F918D
:103918000895689401C0E894309760407040B1F011
:10392800002426F0772312F4009475D1172E7EE137
:10393800112032F07A95EE0FFF1F661F111CF9CF88
:10394800EF2FF62F612D5F938ADF5F9108954F93D4
:10395800AF01FD01DA01AB01BC01CA01402D012C08
:10396800142E4F910895EA0FFB1F681F0895E095E4
:10397800F0956095EF5FFF4F6F4F08955F9381DF7C
:10398800903871F150E8152604C05F937ADF9038BB
:1039980039F1703821F1572F591B2BF112F4D7DF69
:1039A800FACF583118F0AA27BB278827583028F0B3
:1039B800AB2FB82F88275850F9CF552329F0869573
:1039C800B795A7955A95D9F7502D512572F0CBDFA9
:1039D80038F46795F795E795739513F420C0B7DF2A
:1039E8003EDF5F910895D8F7FBCFEA1BFB0B680B0E
:1039F80051F010F40094BBDF662392F3EE0FFF1F23
:103A0800661F7A95CBF7EE27FF27662777275F9102
:103A18000895EFEFFFEF6FE77FEF5F910895EFEF06
:103A2800FFEF6FE77FE75F9108955F932ADF7038B4
:103A380051F3903841F301240894791F23F41CF3BF
:103A480000203AF3ECCF0F921F932F933F934F939D
:103A5800112722279927689FA0018F9F302D410D9C
:103A6800591F6B9F300D411D591F8E9F27D0BF9F37
:103A780025D06A9F23D0BE9F1DD0AF9F1BD0AE9F7D
:103A8800110D291F391F491F591FE32FF42F652FC7
:103A9800522F4F913F912F911F910F9066232AF03B
:103AA800550FEE1FFF1F661F02C073954BF2CDDE48
:103AB8005F910895100D211D391F02C0200D311D81
:103AC800491F591F08955F93DCDE703821F41120D7
:103AD8000AF49FCFA4CF903809F495CF0124089415
:103AE800970B1BF4D4F30020F3CF792F1F932F9358
:103AF8003F934F9311241127222733274427552713
:103B080090E2AE17BF078607410730F0AE1BBF0B28
:103B1800860B410B089401C08894551F221F331F40
:103B2800111CAA1FBB1F881F441F9A9551F7F90142
:103B3800612D4F913F912F911F91662332F0550FC0
:103B4800EE1FFF1F661F7A9543F27FDE5F9108958F
:103B580099239AF0772342F0971748F029F4AE1783
:103B6800BF07860720F031F09894889408959894B8
:103B7800089408951894889408957723C2F797179E
:103B880098F3A9F7EA17FB07680788F399F3ECCFCE
:103B980024975F939F81992311F4289634CF12F4C8
:103BA80028963DCF4F9342E48E81BD81AC818883B6
:103BB8009983AA83BB83FD01BC01AC81BD818E8141
:103BC8009F8181DF88819981AA81BB81DEDE61DEE8
:103BD8007A9545DE88819981AA81BB81AE27A87F25
:103BE80021F4BF178607970729F04A9519F0DF01D6
:103BF800CB01DDCF4F915F91289608950024AF0D3A
:103C0800B01D0895EA0FFB1F681F791F0895F195ED
:103C1800E195F0400895F09560957095E195FF4F16
:103C28006F4F7F4F0895EE0FFF1FEE0FFF1F089590
:103C3800FE2FFF0FFF0B6F2F7F2F08956F2F660F3B
:103C4800660B762F08958B2F880F880B982F089571
:103C5800FA9FF02DEB9FF00DEA9FE02DF10D0895EE
:103C68000024112490E1AA0FBB1F001C111C0E1A7E
:103C78001F0A18F40E0E1F1E01C0A1609A9599F72D
:103C8800FD01D00108953F934F935F9300241124C1
:103C98004427552730E2AA0FBB1F881F991F001C15
:103CA800111C441F551F0E1A1F0A460B570B28F4E8
:103CB8000E0E1F1E461F571F01C0A1603A9559F7E7
:103CC800FD01BC01D001CA015F914F913F91089558
:103CD800C7DFFD010895ED91FC9111970895ED93CB
:103CE800FD936D937C9308950590F491E02D0895CC
:103CF800E881F9816A817B810895A881B9818A81E7
:103D08009B810895E883F9836A837B8308957A9376
:103D18006A93FA93EA930895689401C0E89401D0ED
:103D2800FBDD182E862F612D192E972F712D1B2E36
:103D3800BF2FF12D1A2EAE2FE12D0895129602D025
:103D4800BF011297119602D0FE2F1197E199FECF6D
:103D5800FF93FFB7F894AEBBBFBBE09AEDB3FFBFCC
:103D6800FF91089507D012960F01FB0103D0F001CF
:103D78001297089507D01196EF93EF2F03D0EF9184
:103D880011970895E19B02C0A895FCCF9FB7F894BE
:103D9800AEBBBFBBE09A8DB3E81719F0EDBBE29A52
:103DA800E19A9FBF089530976040704008950024BD
:103DB8000A160B06080609060895EA17FB0768079E
:103DC800790708955A934A933A932A931A930A9330
:103DD80008955D814C813B812A811981088108956C
:00000001FF
